:020000040800F2
:10000000E8310020C1280008E5280008E928000898
:10001000ED280008F1280008F5280008000000007D
:10002000000000000000000000000000F9280008A7
:10003000FD2800080000000001290008F313000853
:1000400005290008092900080D29000811290008C0
:1000500015290008192900081D2900082129000870
:1000600025290008292900082D2900083129000820
:1000700035290008392900083D29000841290008D0
:1000800045290008492900084D2900085129000880
:10009000810E0008CB0E00085529000859290008D8
:1000A0005D29000861290008652900086929000800
:1000B0006D290008712900087529000879290008B0
:1000C0007D29000881290008852900088929000860
:1000D0008D29000891290008952900089929000810
:1000E0009D290008A1290008A5290008A9290008C0
:1000F000AD290008B1290008B5290008000000005A
:10010000B929000800000000BD290008C129000825
:10011000C5290008C9290008CD290008D1290008EF
:10012000D5290008D9290008DD290008E12900089F
:10013000E5290008E9290008ED290008F12900084F
:10014000F5290008F9290008FD290008012A0008FE
:1001500010B5DFF81416884208D140F21944200087
:1001600000F02BFB200000F03BFB07E040F21A44BC
:10017000200000F022FB200000F032FB10BD00291F
:1001800000D1FEE7C0B2002805D002282ED01AD335
:10019000032842D05AE0002048710020C871002096
:1001A000887140F2FF3048810020087200204870BA
:1001B000022088700020C87000200871002048725A
:1001C0000020087070470120C881002008740020BA
:1001D00008810020088000204880002088800020BE
:1001E000C8800020888100204881EBE7002005E0DE
:1001F00000220300DBB20B44DA72401C0200D2B2D0
:10020000082AF5D300208872002048600020087278
:100210000020487200200860D4E7002005E000229A
:100220000300DBB20B44DA72401C0200D2B2082A8F
:10023000F5D300208872002048600020087200205A
:10024000C8740020487200200860BBE7FEE730B4A5
:1002500002000B004FF6FF7001000024156835F016
:1002600002051560156855F00105156000E0491E8E
:10027000151D2D68ED0701D40029F8D1111D09685D
:10028000C90701D400246FE019785D782D0615F0B8
:10029000407555EA81759978090411F470210D4370
:1002A000D978090511F4E0010D435989491E8905E2
:1002B000890D0D4312F11C010D601979012904D13A
:1002C000116851F08001116003E0116831F0800184
:1002D00011605979012904D1116851F04001116070
:1002E00003E0116831F0400111609979012904D1CE
:1002F000116851F02001116003E0116831F0200114
:100300001160D979012904D1116831F0100111600F
:1003100003E0116851F010011160197A012904D12C
:10032000116831F00801116003E0116851F0080113
:100330001160597A012904D1116851F0040111604A
:1003400003E0116831F004011160116849084900A7
:10035000116000E0401E111D0968C90701D5002881
:10036000F8D1002800D001242000C0B230BC704772
:1003700070B400210121428911FA02F2DFF8EC3356
:10038000196851F001011960DFF8E44321689143D5
:100390002160C189002918D1DFF8D8130D68954371
:1003A0000D60C188458855EA01454189DFF8C86379
:1003B00016EBC10635608188058855EA01454189FB
:1003C000DFF8B86316EBC1063560C189012918D181
:1003D000DFF8A0130D6815430D600188458855EAC4
:1003E00001454189DFF8906316EBC10635608188CD
:1003F000C58855EA01454189DFF8806316EBC106DF
:1004000035608189002905D1DFF874130D689543A3
:100410000D6004E0DFF868130D6815430D60018975
:10042000002905D1DFF85C130D6895430D6004E0E9
:10043000DFF850130D6815430D60007C012802D1D0
:10044000206802432260186840084000186070BCB1
:10045000704730B4002210F108021268520101D531
:1004600000220EE010F108021268120101D50122EB
:1004700007E010F108021268D20001D5022200E064
:1004800003221300DBB2032B01D103208FE0130002
:10049000DBB210EB031313F5C0731B6813F00103F9
:1004A0001400E4B210EB041414F5C07423600B7A4A
:1004B000002B13D11300DBB210EB031313F5C07341
:1004C0001B680C684D7A55EA44552B431400E4B27E
:1004D00010EB041414F5C074236014E01300DBB2B5
:1004E00010EB031313F5C0731C684B680D7A55EAC3
:1004F000C3054B7A1D432C431300DBB210EB0313EF
:1005000013F5C0731C601300DBB210EB031313F57B
:10051000C2731B681B091B011400E4B210EB041426
:1005200014F5C27423601300DBB210EB031313F550
:10053000C2731C688B7A1C431300DBB210EB0313ED
:1005400013F5C2731C608B7B4C7B240454EA036458
:100550000B7B54EA0324CB7A1C431300DBB210EB71
:10056000031313F5C4731C608B7C4C7C240454EA85
:1005700003640B7C54EA0324C97B0C431100C9B209
:1005800010EB011111F5C6710C601100C9B210EB2E
:10059000011111F5C071096851F001011300DBB2BE
:1005A00010EB031010F5C07001601000C0B230BC39
:1005B000704700220022C9B2002903D002290DD0C1
:1005C00006D311E008300168DFF8BC0101400CE0FF
:1005D00008300168DFF8B401014006E00830016826
:1005E000DFF8AC01014000E0002100290CD0DFF869
:1005F000980181420AD0DFF89401814208D0DFF8E7
:100600009001814206D007E0022006E0012004E0CC
:10061000012002E0012000E00020C0B270470B0082
:10062000DBB210EB031313F5D8731B6813F004034C
:100630001372137A002B09D10B00DBB210EB0313FA
:1006400013F5D8731B685B0D136008E00B00DBB279
:1006500010EB031313F5D8731B68DB0853600B0012
:10066000DBB210EB031313F5D8731B6813F002030E
:1006700053720B00DBB210EB031313F5DA731B6834
:100680001B0AD3740B00DBB210EB031313F5DA7300
:100690001B6813F00F0393720B00DBB210EB031314
:1006A00013F5DC731B68D3720B00DBB210EB031382
:1006B00013F5DC731B681B0A13730B00DBB210EB22
:1006C000031313F5DC731B681B0C53730B00DBB2B5
:1006D00010EB031313F5DC731B681B0E93730B00F5
:1006E000DBB210EB031313F5DE731B68D3730B003F
:1006F000DBB210EB031313F5DE731B681B0A1374D4
:100700000B00DBB210EB031313F5DE731B681B0C3D
:1007100053740B00DBB210EB031313F5DE731B688D
:100720001B0E9374C9B2002907D110F10C0109689E
:1007300051F020010C30016006E010F11001096851
:1007400051F0200110300160704710F1140212685E
:10075000114314300160704710F11402126832EA3C
:1007600001011430016070470064004000660040E1
:100770001C6600400C660040406600404466004035
:1007800004660040146600400300000400030008F3
:100790000000031010B4DFF87020010009B212EB62
:1007A00091110B68012410F01F018C40234300B20B
:1007B00012EB9012136010BC704710B4DFF84820A1
:1007C000010009B212EB91110B68012410F01F0116
:1007D0008C40234300B212EB9012136010BC7047A0
:1007E00010B4DFF82420010009B212EB91110B685C
:1007F000012410F01F018C40A34300B212EB9012B1
:10080000136010BC70470000001002402DE9F8434F
:10081000040020890B28C0F273810021200000F021
:1008200075FA05000121200000F070FAEDB2552D97
:1008300040F06281C0B2AA2840F05E81022120000F
:1008400000F064FA05000321200000F05FFA0600C2
:100850000421200000F05AFA0700FFB23F020521F0
:10086000200000F053FA57FA80F7EDB2162D04D0AD
:100870000121200000F05FFA42E120893100C9B275
:1008800009318842C0F23C81DFF844545520287079
:10089000AA2068700720A8705120E8703100C9B202
:1008A000083189B2200000F031FAC0B2F0280FD030
:1008B0000121200000F03FFA0120DFF81814087031
:1008C000DFF814044CF202318180F021817017E1CD
:1008D0003100C9B2091D89B2200000F017FA804624
:1008E0003100C9B2491D89B2200000F00FFA8146DB
:1008F0003100C9B2891D89B2200000F007FA5FFA01
:1009000088F85FFA89F95FEA094919EB0869C0B20A
:1009100019EB00293100C9B2C91D89B2200000F0CD
:10092000F5F959FA80F85FF002090AE0494689B200
:10093000200000F0EBF9494689B22944887019F18A
:100940000109484680B23100C9B2091D8842EDDB79
:100950003100C9B2891D89B2280000F022FA804511
:1009600012D00120DFF86C130870DFF86C034CF232
:1009700002318180F1218170F6B20936310089B2ED
:10098000200000F0D8F9BBE0F6B20936310089B298
:10099000200000F0D0F9CF4800214180BFB242F2E0
:1009A00005517F1A00F09D8047F606417F1A07D057
:1009B00040F27A217F1A14D07C3F00F0898096E0C3
:1009C000C5498A78012A0BD001228A70012202705F
:1009D0004CF202428A80D5F80F20CA600021818043
:1009E0008EE0BE4C2078002857D101202070BC4EEC
:1009F00015F10D003060BB49306800F095FA002811
:100A000043D1B949306800F0A0FA306800F0ABFA81
:100A1000002832D1B549306800F0C6FA002824D148
:100A2000306800F0F8FA002817D102202070B04892
:100A300000F036FB002005E00021AE4A03009BB227
:100A4000D154401C010089B2B1F5806FF4DB012163
:100A50004CF2022000F0EEF839E003202070012172
:100A60004CF2023000F0E6F831E003202070012162
:100A70004CF2023000F0DEF829E003202070012162
:100A80004CF2023000F0D6F821E003202070012162
:100A90004CF2023000F0CEF819E02078022816D18E
:100AA0008D480221817015F10D018160A97A09023A
:100AB0006A7A8918491EC180C188B1F5006F01DBCF
:100AC0000021C1804CF2022181800121017017E0D8
:100AD000814903228A70012202704CF20250888000
:100AE0000EE005217C4A91700121017008E001218E
:100AF000200000F020F903E00121200000F01BF9A4
:100B0000BDE8F18370B57C4D1121280000F049F952
:100B10000100090E69740100090CA9740100090A99
:100B2000E9742875754C76480088216808600020B3
:100B300021684872002021680872082021688872A4
:100B400028782168C8726878216808730622291DF0
:100B5000206810F10D06300000F0F2FA206800F075
:100B600043F9002821D0082021688872082215F155
:100B70000A01206810F10B06300000F0E1FA20684D
:100B800000F032F9002810D0042021688872042275
:100B900015F11201206810F10B05280000F0D0FAC1
:100BA000206800F021F90028FFD070BD70B5554CC9
:100BB0000B21200000F0F5F80100090EE1720100A0
:100BC000090C21730100090A6173A0734B4D4C4855
:100BD0000088296808600020296848720020296878
:100BE000087208202968887220782968C87260789D
:100BF000296808730622211D286810F10D063000AF
:100C000000F09EFA286800F0EFF8002811D00620C6
:100C1000296888722868827A14F10A01286810F11C
:100C20000B04200000F08CFA286800F0DDF80028A2
:100C3000FFD070BD70B5344C020092B2120AA2719E
:100C4000E071217289B2090A61720A21200000F064
:100C5000A8F80100090EA1720100090CE17201005F
:100C6000090A21736073254D2548008829680860AA
:100C70000020296848720020296808720820296825
:100C8000887220782968C8726078296808730622FB
:100C9000211D286810F10D06300000F051FA286877
:100CA00000F0A2F8002811D0052029688872286871
:100CB000827A14F10A01286810F10B04200000F078
:100CC0003FFA286800F090F80028FFD070BD0000BF
:100CD00074100020CC110020B0110020E41100207D
:100CE000D811002000000020D4110020E0FF0308EC
:100CF0000030000874080020200000206C00002054
:100D00005800002038000020480000200A00038915
:100D100089B28B4209D3C1888A181100438889B2ED
:100D2000994203D34188521A00E00022C06892B26F
:100D3000805CC0B2704770B504000D0020892900A6
:100D400089B2884216D3734E02213000FFF704FDAA
:100D50002089401B208102213000FFF7F6FCE0884B
:100D600045192800618880B2884201D360882D1A15
:100D7000E58015E0674E02213000FFF7EDFC258984
:100D80000020208102213000FFF7DFFCE0884519B8
:100D90002800618880B2884201D360882D1AE580DE
:100DA00070BD70B400225FF0FF3200250DE05A4B99
:100DB0001600360EF6B253F8263012025A40641C62
:100DC00023009BB2042BF2DB6D1C2B000C009BB2AA
:100DD000A4B2A34205D22B009BB2C35C5A400024AC
:100DE000EEE7100070BC704770B5010000244B4D59
:100DF000484E3000FFF72DFB287000E0641C297876
:100E00003000FFF7D6FB012803D04FF6FF70844275
:100E1000F4D329783000FFF7CCFB4FF6FF70844203
:100E200003D300F079FA002000E0012070BD30B457
:100E300000221DE03A4B1B681400E4B22344DB7A25
:100E4000C4688588635583885B1C83808388448855
:100E5000A34201D30023838003895B1C0381438861
:100E60000489A34203D24388038101238372521C65
:100E700013000C00DBB2E4B2A342DBD330BC7047FA
:100E800038B5244C264D2A6800212000FFF7C7FB07
:100E90002868007A002803D12868807A002804D1C5
:100EA00004212000FFF751FC0EE02868006840F2A2
:100EB0005171884204D12868817A1A48FFF7B7FF38
:100EC00004212000FFF741FC31BD38B5114C144D11
:100ED0002A6800212000FFF7A2FB2868007A00287A
:100EE00003D12868807A002804D104212000FFF76C
:100EF0002CFC0EE02868006840F25171884204D151
:100F00002868817A0748FFF792FF04212000FFF745
:100F10001CFC31BD00640040F81E0008E5110020F3
:100F2000680000205800002030B403000020002595
:100F300000E06D1C102D05DA5A5D4C5D121B002A75
:100F4000F7D0FF20C0B230BC70471CB50C006B4618
:100F500001221349303000F08AFB04226946200048
:100F600000F0EEF813BD3EB5040000256B460022EC
:100F70000C4914F1300000F07AFB002200E0521C12
:100F8000082A09DA6846805C04EB020191F83810FF
:100F9000401A0028F3D0FF252800C0B23EBD000053
:100FA000100000201800002070B488B00200080073
:100FB00000210023002318E010EB8304246825009F
:100FC0002D0E6E4606F8235025002D0C6E4606EBBE
:100FD0008306757025002D0A6E4606EB8306B570F4
:100FE0006D4605EB8305EC705B1C082BE4DB0024ED
:100FF00000E0641C202C09DA02EB040090F8500099
:101000006B461B5DC01A0028F3D0FF210800C0B258
:1010100008B070BC704730B403000020002400E02A
:10102000641C102C12DA0021002504E02A011A4465
:10103000125D51406D1C072DF8DBC9B203EB0402B1
:1010400092F87020891A0029EAD0FF20C0B230BC83
:10105000704730B4002513E050F8042BD30744BF89
:10106000A9F101039A18091F042942F8045BFAD276
:1010700013468C0744BF15809B1CC90748BF1D70D1
:1010800050F8041B0029E7D130BC704780B500F050
:1010900091FB40F2073000F08FFC00F0AEFB01BD89
:1010A00070B505000020002400F084FB00260FE04E
:1010B00009E04FF4006000FB065000F0B3FBC0B243
:1010C0000328F5D1641C40F2073000F075FC761C53
:1010D0004FF4006000FB065017498842E9D300F046
:1010E0008CFB002C01D0012000E0002070BDF8B581
:1010F00004000D001600002000F05CFB002701E05A
:10110000241D7F1CB74212D20C4884420FD255F8DE
:101110002710200000F0F7FB002806D1206855F8C2
:1011200027108842ECD0022004E0032002E000F007
:1011300064FB0020F2BD000000E00308FCDF0308B0
:1011400062B38B0708D0521E11F8013B00F8013B37
:1011500000F024808B07F6D1830740F0208000BF89
:10116000103A07D330B4B1E83810103AA0E838107C
:10117000F9D230BC530724BFB1E80810A0E808102A
:1011800044BF51F8043B40F8043BD20724BF31F878
:10119000022B20F8022B44BF0B7803707047121FFC
:1011A00017D35B0009D151F8043B20F8023B1B0C1C
:1011B000121F20F8023BF6D20BE051F8043B00F876
:1011C000013B1B0A20F8023B1B0C121F00F8013BDD
:1011D000F3D238BF121D521E24BF11F8013B00F894
:1011E000013BF8D870470000020052B2002A08D52F
:1011F00009019E4A40B210F00F00104400F8041C90
:1012000003E009019A4A40B21154704780B5411E6B
:10121000B1F1807F01D301200EE0401E95490860A6
:101220000F215FF0FF30FFF7DFFF002092490860D9
:10123000072092490860002002BD80B500F011F837
:1012400000F029F801BD80B500F005F800F0D7F8EE
:1012500000F0E5F801BD80B500F0B3F800F05CF8EF
:1012600001BD80B54FF4C060FFF794FA40F2026010
:10127000FFF790FA40F20360FFF78CFA40F2046047
:10128000FFF788FA40F20760FFF784FA40F219701E
:10129000FFF780FA01BD10B5794C4FF4805303225B
:1012A0001021200000F000FC4FF48051200000F0DD
:1012B0006DFC4FF4004303224821200000F0F4FBB2
:1012C0004FF40041200000F061FC01215FF4EA10BE
:1012D00000F05FFC6B4C4FF480730322042120006C
:1012E00000F0E2FB4FF4007303221821200000F00D
:1012F000DBFB654C022303221021200000F0D4FB0D
:101300000221200000F03FFC4FF401430322102192
:10131000200000F0C9FB10BD10B588B06946002060
:10132000FEF72DFF03A90020FEF729FF574C2000F0
:10133000FEF70EFF00208DF8040001208DF8050057
:1013400000208DF8060001208DF8070000208DF8A0
:10135000080001208DF8090000208DF80000002011
:101360008DF8010005208DF8020000208DF80300A3
:101370001220ADF80A0069462000FEF768FF002041
:10138000ADF816000020ADF818000120ADF81A00E5
:101390004EF62020ADF80C000020ADF80E004FF600
:1013A000E070ADF810000020ADF812000020ADF89C
:1013B000140001208DF81C0003A8FEF7D9FF08B027
:1013C00010BD80B5324800684FF47A71B0FBF1F07F
:1013D000FFF71CFF01BD2F49086008680028FCD1F9
:1013E00070472C490868002802D00868401E086031
:1013F000704780B5FFF7F5FF00F000FD01BD80B537
:101400004FF4A06000F016FD00220321142000F02C
:1014100016FD00220321152000F011FD01BD10B5BD
:101420001A4C02212000FFF790F908212000FFF755
:101430008CF910212000FFF788F940212000FFF7E8
:1014400084F94FF400412000FFF77FF94FF48061E9
:101450002000FFF77AF94FF480712000FFF775F94B
:101460004FF400712000FFF770F910BD18ED00E097
:1014700000E400E014E000E018E000E010E000E02C
:1014800000080140000C01400010014000640040D1
:1014900070000020DC110020F0B4BB4D00240026B9
:1014A0000E55641C082CFADB00261478521C270009
:1014B000FF10C75D14F007042C5D274209D03400EB
:1014C000E4100F5D16F007042C5D27433400E41090
:1014D0000F55761C1C00E4B2A642E6DBF0BC704758
:1014E0001CB4002107E00A00D2B2825C6B460C00FB
:1014F000E4B21A55491C0A00D2B2082AF3DB0021D3
:101500001AE00A00D2B2825C52000B00DBB2C25475
:101510000A00D2B2062A0EDA6A460B00DBB21A447F
:101520005278120607D50A00D2B2825C52F001024C
:101530000B00DBB2C254491C0A00D2B2072AE0DB1E
:101540009DF80010090604D5C17851F01001C17052
:1015500003E0C17811F0EF01C1709DF80310090795
:1015600004D5817951F00101817103E0817911F095
:10157000FE01817113BC704738B584B0002107E0CB
:101580000A00D2B2825C814B0C00E4B21A55491CAD
:101590000A00D2B2082AF3DB38237D4A6946FFF7F6
:1015A0007BFF002411E07B492200D2B201EBC20193
:1015B0000200D2B202AB0500EDB25B5D8B54401C61
:1015C0000100C9B20829EEDB641C2000C0B210285B
:1015D00015DA002503E06846FFF782FF6D1C28003E
:1015E0006D492200D2B2895CC0B28842F3D3402355
:1015F0006A4A02A96846FFF74FFF0020E0E705B0FE
:1016000030BD70B586B00400080015004023644A60
:1016100002A9FFF741FF00211DE004AA02A80B0068
:10162000DBB2C35C0800C0B2205C434013F03F0350
:101630000800C0B213545B4B0E00F6B24020464384
:1016400003EB06000B00DBB2D25C805C6A460B0049
:10165000DBB2D054491C0800C0B20828DDDB2023CF
:10166000514A29006846FFF717FF06B070BDF8B56C
:1016700086B006000F0015001C0000200DE00100E0
:10168000C9B2795C414A0300DBB2D25C914203D01B
:101690003800FFF771FF0720401C0100C9B208297C
:1016A000EDDB4023414A69463000FFF7F5FE012695
:1016B00013E002A80A00D2B2825C04A80B00DBB2DD
:1016C000C05C424068460B00DBB218440271491C02
:1016D0000800C0B20428ECDB761C3000C0B2112830
:1016E00036DA002008E069460200D2B2895C02AA1C
:1016F0000300DBB2D154401C0100C9B20829F2DB5F
:101700002800C0B2002806D122483100C9B200EB3F
:10171000C100083806E01F483100C9B2494200EB59
:10172000C1008030002109E002AA0B00DBB21A449C
:1017300012796B460F00FFB2DA55491C0A00D2B28B
:10174000042AF1DB04AA6946FFF75BFF0021BFE72B
:101750009DF8000069460A798DF8002008714878E4
:101760004A794A70487188788A798A708871C8780D
:10177000CA79CA70C87140230D4A21006846FFF734
:101780008BFE07B0F0BD0000DC280008C41100206B
:101790005427000808110020B0280008D4260008AB
:1017A00014270008F82200083028000854260008F2
:1017B00094260008DFF86C020068000607D5DFF801
:1017C0006802DFF868120160DFF864120160DFF878
:1017D0006402008880B240F2012188420CD3DFF815
:1017E00058020068000607D5DFF85002DFF83C1207
:1017F0000160DFF83C1201607047DFF828020168E1
:1018000051F080010160DFF82C02008880B240F2C4
:101810000121884205D3DFF82002016851F08001E0
:101820000160704770B50400DFF80802008880B2DC
:1018300040F20121884247D3DFF8040284421DD2DE
:10184000DFF80052280000F009F90100C9B20029B0
:1018500057D1DFF8D061306850F002003060DFF817
:10186000E8010460306850F040003060280000F06B
:10187000F5F8316831F00201316042E0DFF8C4511F
:10188000280000F0FEF80100C9B2002939D1DFF8C4
:10189000A861306850F002003060DFF8B0010460E9
:1018A000DFF8AC010068800702D5DFF89C01046016
:1018B000306850F040003060280000F0E2F83168F5
:1018C00031F0020131601CE0DFF87851280000F0AF
:1018D000C5F80100C9B2002913D1DFF848613068AA
:1018E00050F002003060DFF860010460306850F0B2
:1018F00040003060280000F0B1F8316831F002019A
:101900003160C0B270BDF8B504000D000020DFF8F2
:101910002401008880B240F20121884233D3DFF8ED
:101920002001844217D2DFF81C61300000F096F8E5
:101930000100C9B200293DD1DFF8E870386850F0E5
:10194000010038602560300000F088F839684908E7
:10195000490039602EE0DFF8EC60300000F091F8CB
:101960000100C9B2002925D1DFF8CC70386850F0E9
:10197000010038602560300000F083F839684908BC
:101980004900396016E0DFF8BC60300000F066F80E
:101990000100C9B200290DD1DFF88870386850F015
:1019A000010038602560300000F058F839684908B7
:1019B00049003960C0B2F2BD10B4194A12EB90115F
:1019C0000B68012410F01F018C40234312EB90128E
:1019D000136010BC704700201E490A68D20701D569
:1019E000012008E00A68D20601D5032003E0096857
:1019F000490700D50220C0B27047002016490A6886
:101A0000D20701D5012008E00A68D20601D50320DB
:101A100003E00968490700D50220C0B27047000002
:101A200000200240102002400420024023016745AC
:101A3000AB89EFCDE0F7FF1F502002404420024069
:101A4000FFFF07080000FF0F14200240542002404F
:101A50001C2002400C2002404C20024010B5040023
:101A60000120FFF7B8FF641E0100C9B2012901D1AE
:101A7000002CF6D10100C9B2012900D10420C0B266
:101A800010BD10B504000120FFF7B7FF641E010070
:101A9000C9B2012901D1002CF6D10100C9B2012936
:101AA00000D10420C0B210BDF0B40024002411F015
:101AB0000F04CD060DD5042A09D154F0030410F10A
:101AC0003C0212681A4310F13C052A6001E02243EF
:101AD0001400002523E048291FD10122AA401A4002
:101AE00010F110073A6018E01A00EA40D20715D545
:101AF00006680F272A00D2B292009740BE432A0000
:101B0000D2B2920014FA02F216432829E3D101223C
:101B1000AA401A4010F114073A6006606D1C2A00B2
:101B200092B2082AE0D3082527E0482922D10122D1
:101B3000AA401A4010F110073A601BE01A00EA4070
:101B4000D20719D5021D16680F272A00083AD2B20B
:101B500092009740BE432A00083AD2B2920014FA8B
:101B600002F216432829E0D10122AA401A4010F1BE
:101B700014073A60021D16606D1C2A0092B2102AEA
:101B8000DCD3F0BC70471030016070471430016046
:101B9000704730B40022002200220022002802D523
:101BA0001E4A146801E01E4A1468C0F3034283B25F
:101BB00010F44015B5F5401F08D1220032F0E06264
:101BC000174C256835F0E065256013E0C50207D5A0
:101BD000032515FA02F234EA020252F0E06209E04B
:101BE0000200520DD2B2120113FA02F234EA0202DA
:101BF00052F0E062C9B2002906D00100490DC9B215
:101C000009018B4013431A00002802D503480260E3
:101C100001E00348026030BC704700001C00014036
:101C20000400014001B582B0029801687748014084
:101C3000B1F1005F0DD10298001D0068009074485A
:101C4000009901600299096881F30888006880475B
:101C500002E00120FFF7BFFB07BD80B5FFF716FAD2
:101C60006C48002181700021C18000210170002199
:101C700041700021017468484FF47A71818000211D
:101C8000418001BD80B56548FEF7C0FD00F02EF82B
:101C900000F043F800F012F85E4840780128F2D1D5
:101CA0003220FFF798FB5E48FEF752FA02215D48AA
:101CB000FFF76CFF5C48FFF7B5FFE4E710B5554C44
:101CC0006078002811D1A07800280ED052484188B1
:101CD00040F6B932914208DB00214180E1884CF2A4
:101CE0000230FEF7A7FF0120607010BD80B54949A2
:101CF0008878002810D1087C04280BDA46488288AE
:101D0000322A09DB00228280087C401C0874FEF71E
:101D1000F9FE01E00120487001BDF8B53E4C207885
:101D2000012826D1002020703A4DA878012806D03D
:101D3000022809D003280CD0052811D019E0002171
:101D4000A888FEF777FF14E0E988A888FEF772FFFD
:101D50000FE00021A888FEF76DFF0120687008E001
:101D6000FEF724FF0020A87000206870002028746F
:101D7000FFE7284D287801283FD100202870E88807
:101D800040F60101884233DAE888002830D0274E37
:101D9000E888304410F8010C00281ED12022A968E0
:101DA000E8888027224B07FB0030FFF7A0F90028C6
:101DB00009D0EE214CF20260FEF73CFF4FF47A703E
:101DC000FFF709FBF5E70120E988314401F8010C30
:101DD00001202070002060800FE0E9884CF2022092
:101DE000FEF728FFE1214CF20260FEF723FF04E03A
:101DF000E2214CF20260FEF71DFFF1BD064881882A
:101E0000491C81804188491C418070470000FE2F99
:101E1000E0110020B0110020CC110020580000205B
:101E200000640040001001400030000874080020E9
:101E3000802F00082C4908432C490860704770B572
:101E400004000D0016000020002000202748016833
:101E500011F4E061B1F5E06F02D10020042129E026
:101E6000016811F4E061B1F5C06F02D101200321D6
:101E700020E0016811F4E061B1F5A06F02D1022009
:101E8000022117E0016811F4E061B1F5806F02D121
:101E9000032001210EE0006810F4E060B0F5407FFF
:101EA00002D10420002105E04FF4A060FFF7C2FF3B
:101EB00002200221EDB2D0F104008540F6B20F20DD
:101EC000D1F10401C840064035432D0108482100E6
:101ED000C9B24554012114F01F0081400548E4B205
:101EE000641140F8241070BD0000FA050CED00E00C
:101EF00000E400E000E100E000000000B71DC104C4
:101F00006E3B8209D926430DDC7604136B6BC51733
:101F1000B24D861A0550471EB8ED08260FF0C922AB
:101F2000D6D68A2F61CB4B2B649B0C35D386CD3113
:101F30000AA08E3CBDBD4F3870DB114CC7C6D048DF
:101F40001EE09345A9FD5241ACAD155F1BB0D45BBB
:101F5000C2969756758B5652C836196A7F2BD86E23
:101F6000A60D9B6311105A6714401D79A35DDC7D9B
:101F70007A7B9F70CD665E74E0B6239857ABE29C87
:101F80008E8DA191399060953CC0278B8BDDE68FBB
:101F900052FBA582E5E66486585B2BBEEF46EABAA3
:101FA0003660A9B7817D68B3842D2FAD3330EEA99B
:101FB000EA16ADA45D0B6CA0906D32D42770F3D0FF
:101FC000FE56B0DD494B71D94C1B36C7FB06F7C333
:101FD0002220B4CE953D75CA28803AF29F9DFBF62B
:101FE00046BBB8FBF1A679FFF4F63EE143EBFFE513
:101FF0009ACDBCE82DD07DEC77708634C06D47302B
:10200000194B043DAE56C539AB0682271C1B432332
:10201000C53D002E7220C12ACF9D8E1278804F16AA
:10202000A1A60C1B16BBCD1F13EB8A01A4F64B0512
:102030007DD00808CACDC90C07AB9778B0B6567CDE
:1020400069901571DE8DD475DBDD936B6CC0526FBA
:10205000B5E6116202FBD066BF469F5E085B5E5A22
:10206000D17D1D576660DC5363309B4DD42D5A499A
:102070000D0B1944BA16D84097C6A5AC20DB64A84E
:10208000F9FD27A54EE0E6A14BB0A1BFFCAD60BBBA
:10209000258B23B69296E2B22F2BAD8A98366C8EA2
:1020A00041102F83F60DEE87F35DA9994440689D9A
:1020B0009D662B902A7BEA94E71DB4E0500075E4FE
:1020C000892636E93E3BF7ED3B6BB0F38C7671F732
:1020D000555032FAE24DF3FE5FF0BCC6E8ED7DC22A
:1020E00031CB3ECF86D6FFCB8386B8D5349B79D112
:1020F000EDBD3ADC5AA0FBD8EEE00C6959FDCD6D80
:1021000080DB8E6037C64F643296087A858BC97E35
:102110005CAD8A73EBB04B77560D044FE110C54BA5
:10212000383686468F2B47428A7B005C3D66C15815
:10213000E4408255535D43519E3B1D252926DC21F9
:10214000F0009F2C471D5E28424D1936F550D832BD
:102150002C769B3F9B6B5A3B26D6150391CBD4071D
:1021600048ED970AFFF0560EFAA011104DBDD0149D
:10217000949B93192386521D0E562FF1B94BEEF501
:10218000606DADF8D7706CFCD2202BE2653DEAE6BD
:10219000BC1BA9EB0B0668EFB6BB27D701A6E6D39D
:1021A000D880A5DE6F9D64DA6ACD23C4DDD0E2C09D
:1021B00004F6A1CDB3EB60C97E8D3EBDC990FFB9D9
:1021C00010B6BCB4A7AB7DB0A2FB3AAE15E6FBAA35
:1021D000CCC0B8A77BDD79A3C660369B717DF79F25
:1021E000A85BB4921F4675961A163288AD0BF38C15
:1021F000742DB081C330718599908A5D2E8D4B59B5
:10220000F7AB085440B6C95045E68E4EF2FB4F4A34
:102210002BDD0C479CC0CD43217D827B9660437FA4
:102220004F460072F85BC176FD0B86684A16476C14
:1022300093300461242DC565E94B9B115E565A15F8
:1022400087701918306DD81C353D9F0282205E06BC
:102250005B061D0BEC1BDC0F51A69337E6BB52331C
:102260003F9D113E8880D03A8DD097243ACD56209C
:10227000E3EB152D54F6D4297926A9C5CE3B68C1C8
:10228000171D2BCCA000EAC8A550ADD6124D6CD2BC
:10229000CB6B2FDF7C76EEDBC1CBA1E376D660E79C
:1022A000AFF023EA18EDE2EE1DBDA5F0AAA064F49C
:1022B000738627F9C49BE6FD09FDB889BEE0798DD8
:1022C00067C63A80D0DBFB84D58BBC9A62967D9E34
:1022D000BBB03E930CADFF97B110B0AF060D71AB24
:1022E000DF2B32A66836F3A26D66B4BCDA7B75B814
:1022F000035D36B5B440F7B10E040D01020F0B08B3
:10230000030A060C05090007000F07040E020D0161
:102310000A060C0B0905030804010E080D06020B42
:102320000F0C0907030A05000F0C08020409010736
:10233000050B030E0A00060D0F01080E060B030421
:102340000907020D0C00050A030D04070F02080E11
:102350000C00010A06090B05000E070B0A040D010B
:1023600005080C060903020F0D080A01030F0402F9
:102370000B06070C00050E090A00090E06030F05DF
:10238000010D0C070B0402080D0700090304060ADF
:102390000208050E0C0B0F010D060409080F0300BF
:1023A0000B01020C050A0E07010A0D0006090807B9
:1023B000040F0E030B05020C070D0E030006090A9D
:1023C000010208050B0C040F0D080B05060F000396
:1023D0000407020C010A0E090A0609000C0B070D7E
:1023E0000F01030E05020804030F00060A010D0881
:1023F0000904050B0C07020E020C0401070A0B0668
:102400000805030F0D000E090E0B020C04070D0149
:1024100005000F0A030908060402010B0A0D07084C
:102420000F090C050603000E0B080C07010E020D28
:10243000060F00090A0405030C010A0F0902060829
:10244000000D03040E07050B0A0F0402070C090513
:1024500006010D0E000B0308090E0F0502080C0300
:102460000700040A010D0B060403020C09050F0AFC
:102470000B0E01070600080D040B020E0F00080DDD
:10248000030C0907050A06010D000B070409010AE0
:102490000E03050C020F080601040B0D0C03070EBA
:1024A0000A0F060800050902060B0D0801040A07B9
:1024B0000905000F0E02030C0D020804060F0B01A4
:1024C0000A09030E05000C07010F0D080A03070493
:1024D0000C05060B000E0902070B0401090C0E0285
:1024E00000060A0D0F03050802010E07040A080D75
:1024F0000F0C09000305060B80B54B48016851F429
:10250000700101604949086850F0010008600868DE
:102510008007FCD5464A106850F08000106000200B
:10252000009002E00098401C009000985028F9D3D9
:10253000106850F0900010600020009002E00098B9
:10254000401C009000985028F9D310688008800043
:1025500010600B68374803400B605FF47F00364B18
:102560001860086830F480200860002010600020A7
:102570003249086000F001F801BD80B500F001F8B3
:1025800001BD10B4002200202849086850F0010065
:102590000860521C086810F00200002802D1B2F551
:1025A000A06FF6D10868800700D4FEE724480268CF
:1025B00052F080520260234A106850F4404010608C
:1025C0001B4B1868186018681860186850F4806011
:1025D00018601C681C4804401C601C681B480443AD
:1025E0001C60086850F08070086008688001FCD5A5
:1025F000106850F48030106015480168C903FBD59D
:10260000116851F40031116001688903FCD5186824
:10261000800880001860186850F002001860186880
:102620000007FCD510BC704788ED00E000100240A8
:1026300004100240FFFFF6EA081002402C1002408E
:102640001C10024000700040FFFFC39F00000420E8
:102650000470004039312921191109013B332B2322
:102660001B130B033D352D251D150D053F372F275A
:102670001F170F0738302820181008003A322A2276
:102680001A120A023C342C241C140C043E362E264A
:102690001E160E0627072F0F37173F1F26062E0E72
:1026A00036163E1E25052D0D35153D1D24042C0C1A
:1026B00034143C1C23032B0B33133B1B22022A0A2A
:1026C00032123A1A2101290931113919200028083A
:1026D0003010381800000D04100A1700000002091D
:1026E0001B0E051400001607120B031900000F0142
:1026F000061A130C00002836331E242E00001D2F4E
:1027000027322C2000002B343026372100002D1FCB
:102710002931231C00001F040001020300000308EC
:10272000040506070000070C08090A0B00000B103F
:102730000C0D0E0F00000F141011121300001318CF
:10274000141516170000171C18191A1B00001B007F
:102750001C1D1E1F3830282018100800393129216F
:10276000191109013A322A221A120A023B332B2389
:102770003E362E261E160E063D352D251D150D0541
:102780003C342C241C140C041B130B0330B50168BF
:1027900084684218416802EB5103C90703D54C44D1
:1027A00001E0491C05D19A420AD012F9011B12F826
:1027B000015B002904F8015BF3D4491EF7D5F2E769
:1027C0000C3030BD10B5074979441831064C7C44B3
:1027D000163404E00A68081D114488470146A142E6
:1027E000F8D110BD2C000000480000004EF68851C2
:1027F000CEF20001086840F470000860BFF34F8F0C
:10280000BFF36F8F4FF00070E1EE100A70470000C9
:1028100043E8FFFF74110000740000200000000076
:102820006DFFFFFFE0010000D2000000000000206B
:102830001F0E272C3C173724041E2E350C253E1561
:10284000050F2F1D3F360614261C3D0D2D1607348F
:1028500000F00DF8002801D0FFF7B4FFAFF30080BF
:102860000020AFF3008000F004F800F00EF8012023
:10287000704780B572B6FEF7E0FCFEF7E4FC62B686
:10288000FFF7EBF9FFF7FEF9FEE700F001B80000F3
:102890000746384600F002F8FBE7000080B5AFF3CA
:1028A0000080024A11001820ABBEFBE726000200A0
:1028B00001010202020202020102020202020201FC
:1028C0000148804701480047F9240008D128000842
:1028D000AFF30080FFF78AFFFFF7BAFF80402010B8
:1028E00008040201FFF7FEBFFFF7FEBFFFF7FEBFC0
:1028F000FFF7FEBFFFF7FEBFFFF7FEBFFFF7FEBF0C
:10290000FFF7FEBFFFF7FEBFFFF7FEBFFFF7FEBFFB
:10291000FFF7FEBFFFF7FEBFFFF7FEBFFFF7FEBFEB
:10292000FFF7FEBFFFF7FEBFFFF7FEBFFFF7FEBFDB
:10293000FFF7FEBFFFF7FEBFFFF7FEBFFFF7FEBFCB
:10294000FFF7FEBFFFF7FEBFFFF7FEBFFFF7FEBFBB
:10295000FFF7FEBFFFF7FEBFFFF7FEBFFFF7FEBFAB
:10296000FFF7FEBFFFF7FEBFFFF7FEBFFFF7FEBF9B
:10297000FFF7FEBFFFF7FEBFFFF7FEBFFFF7FEBF8B
:10298000FFF7FEBFFFF7FEBFFFF7FEBFFFF7FEBF7B
:10299000FFF7FEBFFFF7FEBFFFF7FEBFFFF7FEBF6B
:1029A000FFF7FEBFFFF7FEBFFFF7FEBFFFF7FEBF5B
:1029B000FFF7FEBFFFF7FEBFFFF7FEBFFFF7FEBF4B
:1029C000FFF7FEBFFFF7FEBFFFF7FEBFFFF7FEBF3B
:1029D000FFF7FEBFFFF7FEBFFFF7FEBFFFF7FEBF2B
:1029E000FFF7FEBFFFF7FEBFFFF7FEBFFFF7FEBF1B
:1029F000FFF7FEBFFFF7FEBFFFF7FEBFFFF7FEBF0B
:102A0000FFF7FEBF30AE7AE501B6B24B678758D804
:102A10006C69E8E5FE4D4F54494E4F564141564FC3
:102A20004E49544F4D55AA07150C0BC1094D432073
:102A300056322E352E30FC000DF0000055AA071539
:102A40000C05A90341434BFC0006F055AA07150CE1
:102A500004F80005F00015070008F8000F740000E6
:0D2A600020881100209C11002000A24A04D3
:04000005080028D1F6
:00000001FF
